:100000008316043085000030860083129C00A628E9
:1000100082070334073406340434023406340734C8
:100020000334053402340234033405340434023416
:1000300007340634073404340334023405340734F7
:1000400006340334023402340334043405340434F3
:1000500003340734043406340734023403340434DC
:100060000534013400309100083092001C309300B8
:10007000083094000030950074280330910003305C
:100080009200003093006030940060309500742836
:10009000033091000B3092001C30930068309400C4
:1000A0006030950074286330910063309200003016
:1000B000930063309400633095007428633091009E
:1000C0006B3092001C3093006B30940063309500CD
:1000D00074286B3091006B309200003093006B30CD
:1000E00094006B3095007428851400008510110869
:1000F0008600872012088600872013088600872044
:1001000014088600872015088600872008009B0BAE
:1001100087280030860005140000051008001C0820
:1001200008209D009D0B972800309C008F289D0B78
:100130009A2832289D0B9D283D289D0BA0284828F1
:100140009D0BA32853289D0B69285E2830308C0016
:100150008F208C0BA8289C0A40308C008F208C0BA1
:10016000AE289C0A50308C008F208C0BB4289C0A3F
:1001700060308C008F208C0BBA289C0A70308C0069
:100180008F208C0BC0289C0A8F20051DC428A62810
:00000001FF
